:020000040000FA
:100000000B28200882073834383438343834013427
:100010000C34063400348316030185008700003059
:10002000890013308600F03088008312303094004D
:1000300085018601870188018901B501A001891424
:10004000B621E1218A01EE218A01BD22BD22D22101
:10005000FC218A01BD22BD22D2218630CF212E3043
:10006000C921D6218B210F30B800FF30B9006D2097
:100070000A128A159E218A110130A4000A128A15DB
:10008000E8200430A5000A128A152F2162210F22D0
:1000900047289E208A1500200800EF208A1500209E
:1000A00008003710B90F6D28B80A10303802031D48
:1000B0006D280F30B800FF30B9006D2808003718E0
:1000C0000800B90B6D28B80BFF303802031D6D28EE
:1000D000B801B90137146D28080005300A22B808A4
:1000E0000A22B9080A220F30380503190800D62160
:1000F0003808BA00C0303A07CF21FF30C921BA0B07
:100100007A280800A50A0B302502031D8B288828B1
:100110000A30A50008000A128A152F216221080062
:10012000A50303012502031D992896280130A50087
:1001300008000A128A152F216221080001302402CA
:100140000319AF28023024020319B6280330240211
:100150000319BD28043024020319C428CB283930E0
:100160002C06031DDA283030AC003F21393026063A
:10017000031DDD283030A600442139302706031D39
:10018000E0283030A700492139302806031DE32834
:100190003030A8004E2139302906031DE6283030C2
:1001A000A900532139302A06031DE9283030AA005E
:1001B0005821EC28AC0A3F210800A60A4421080077
:1001C000A70A49210800A80A4E210800A90A5321BC
:1001D0000800AA0A58210800AB0A5D210800013076
:1001E00024020319002902302402031907290330CD
:1001F000240203190E2904302402031915291C298D
:1002000030302C02031D2D293930AC003F21303015
:100210002602031D30293930A60044213030270240
:10022000031D33293930A700492130302802031D2E
:1002300036293930A8004E2130302902031D3929D2
:100240003930A900532130302A02031D3C293930AE
:10025000AA005821AB035D210800AC033F21080030
:10026000A60344210800A70349210800A8034E2142
:100270000800A90353210800AA0358210800883068
:10028000CF212C08C92108008730CF212608C92199
:1002900008008530CF212708C92108008430CF21EC
:1002A0002808C92108008330CF212908C921080066
:1002B0008230CF212A08C92108008130CF212B08A4
:1002C000C92108003F21442149214E2153215821B1
:1002D0005D218A1500208A110800313094008910B0
:1002E0000230A0000A223208A0000A223108A00031
:1002F0000A223008A0000A222F08A0000A222E0895
:10030000A0000A222D08A0000A220914091089144D
:1003100030309400080031309400AD01AE01AF01DF
:10032000B001B101B2010915B622091189100914F1
:100330000000091007300A2214300A2222300A2253
:1003400001300A2240300A2205300A2200300A22F7
:1003500000300A2200300A220A300A220914000062
:1003600009108914303094006D2108009E22061176
:10037000012000380319C22986150A2286119E22FF
:10038000A00AB8290800061186150A228611A6229D
:100390000800061586150A228611AA220800C32124
:1003A000061508008030CF21DA210800C030CF21A7
:1003B000DA2108001030A0002030C921A00BDC2970
:1003C00008008430CF21A0010D308A0000250038BC
:1003D000031908008A01C921A00AE429C230CF21EB
:1003E000A0010D308A000C250038031908008A018D
:1003F000C921A00AF12908008230CF21A0010D30C7
:100400008A001B250038031908008A01C921A00AA7
:10041000FF2908008C1193008C1D0C2A0800722201
:10042000003023020319522A013023020319552AEE
:100430000230230203195A2A0330230203195C2ACB
:100440000430230203195E2A053023020319612AAE
:10045000063023020319662A073023020319682A8B
:100460000830230203196A2A0930230203196B2A70
:100470000A30230203196C2A0B30230203196D2A58
:100480000C30230203196E2A0D30230203196F2A40
:100490000E3023020319702A0F3023020319712A28
:1004A0008A0108008220B92208008A15BF208A111B
:1004B000B922080049200800512008009020B922E4
:1004C00008008A15C9208A11B92208004D200800A9
:1004D0005F20080008000800080008000800080065
:1004E00008000800782210302302031823080800AF
:1004F000A30188010430A2000314880D0310081A18
:100500008D2AA30A881A8D2AA30A081B8D2AA30AFA
:10051000881B8D2AA30AA20B7D2A0800FF308316B0
:10052000D000AD2A80308316D000AD2A403083162B
:10053000D000AD2A20308316D000AD2A10308316AB
:10054000D000AD2A05308316D000AD2A02308316C4
:10055000D000AD2A01308316D000FF308316D100C1
:10056000D10BB02AD00BAD2A831208008E228E2226
:1005700008008E228E228E2208008E228E228E224B
:040580008E220800BF
:10100000B401AD01AE01AF01B001B101B20183166F
:101010002608A0002708A1002808A2002908A3008C
:101020002A08A4002B08A500831230302C020319D3
:101030001B28B400982083162C08A0002D08A100BE
:101040002E08A2002F08A3003008A4003108A50034
:1010500083123030260203192F28B40098208316FB
:101060003208A0003308A1003408A2003508A3000C
:101070003608A4003708A500831230302702031970
:101080004328B400982083163808A0003908A1002E
:101090003A08A2003B08A3003C08A4003D08A500B4
:1010A00083123030280203195728B4009820831681
:1010B0003E08A0003F08A1004008A2004108A3008C
:1010C0004208A4004308A500831230302902031906
:1010D0006B28B400982083164408A0004508A1009E
:1010E0004608A2004708A3004808A4004908A50034
:1010F000831230302A0203197F28B4009820831607
:101100004A08A0004B08A1004C08A2004D08A3000B
:101110004E08A4004F08A500831230302B02031C98
:10112000952803199528B40098208A016D2108009C
:101130009C20B40B98280800831620088312AD0762
:10114000831621080318210F8312AE078316220885
:101150000318220F8312AF07831623080318230FE7
:101160008312B007831624080318240F8312B107D3
:10117000831625080318250F8312B2070800A40A56
:1011800006302402031DC728C5280530A400D3203B
:101190000800A40303012402031DD128CF28013035
:1011A000A400D3200800013024020319E8200230F3
:1011B00024020319F7200330240203190621043006
:1011C00024020319132105302402031920210800E9
:1011D0008A018930CF212030C9212030C921313006
:1011E000C9213030C9214830C9218A0108008A014B
:1011F0008930CF212030C9213130C9213030C92177
:101200003030C9214830C9218A0108008A018A305A
:10121000CF212030C9212030C9213130C9216B3084
:10122000C9218A0108008A018A30CF212030C921D2
:101230003130C9213030C9216B30C9218A01080001
:101240008A018A30CF212030C9213130C921303084
:10125000C9213030C9216B30C9218A010800013011
:101260002502031955290230250203195A29033092
:10127000250203195F29043025020319642905306A
:101280002502031969290630250203196E29073042
:10129000250203197329083025020319782909301A
:1012A000250203197D29822908000030B600872114
:1012B0008A0108000830B60087218A010800103032
:1012C000B60087218A0108001830B60087218A01FC
:1012D00008002030B60087218A0108002830B600B7
:1012E00087218A0108003030B60087218A01080072
:1012F0003830B60087218A0108004030B6008721C7
:101300008A0108004830B60087218A0108000A12C5
:101310008A15FE21AB00B60AFE21AA00B60AFE21FC
:10132000A900B60AFE21A800B60AFE21A700B60A47
:10133000FE21A600B60AFE21AC000800B6018D0110
:101340005030B600FE218316A600F921A700F9212E
:10135000A800F921A900F921AA00F921AB00F9217F
:10136000AC00F921AD00F921AE00F921AF00F9215F
:10137000B000F921B100F921B200F921B300F9213F
:10138000B400F921B500F921B600F921B700F9211F
:10139000B800F921B900F921BA00F921BB00F921FF
:1013A000BC00F921BD00F921BE00F921BF00F921DF
:1013B000C000F921C100F921C200F921C300F921BF
:1013C000C400F921C500F921C600F921C700F9219F
:1013D000C800F921C900F921CA00F921CB00F9217F
:1013E000CC00F921CD00F921CE00F921CF008312E4
:1013F00008008312B60AFE21831608003608031778
:1014000083128D0083168C130C1483120C080313A3
:1014100008003608031783128D00031333080317DF
:101420008C0083168C130C1555308D00AA308D005E
:0A1430008C140C1183120313080042
:101A0000200882074234493445344E345634453434
:101A10004E34553421340034200882074834413490
:101A20004D342034473445344E3445342034353435
:101A3000323421340034200882072034203420340A
:101A400046343634453448344A3420342034203443
:021A5000003460
:02400E00723707
:104200002000310038003000300030003000200045
:104210002000330037003000300030003000200034
:104220002000370030003400300030003000200023
:10423000310030003000300030003000300020000D
:1042400031003400310030003000300030002000F8
:1042500031003800310031003000300030002000E3
:1042600032003100310035003000300030002000D5
:1042700032003400390033003000300030002000BC
:1042800032003800350030003000300030002000AF
:1042900035003000310030003000300030002000A8
:1042A0009400BF00D600000000000000D0007B009A
:1042B00063000800000000002300D600E200530065
:1042C0000000000063005D00DC0046000300000009
:1042D000E300A5009B00C40020000000E1007A007C
:1042E0001400AE0047000100CC00CC00CC00CC0094
:0442F000CC000C00F2
:0A43E60046003600450048004A007A
:0C43F00020005600350032003900390072
:00000001FF
